:10000000D80001207506000071060000710600008E
:10001000710600007106000071060000000000007B
:100020000000000000000000000000007106000059
:10003000710600000000000071060000710600005B
:1000400071060000710600007106000071060000D4
:1000500071060000710600007106000071060000C4
:1000600071060000710600007106000071060000B4
:1000700071060000710600007106000071060000A4
:100080007106000071060000710600007106000094
:100090007106000071060000710600007106000084
:1000A0007106000071060000710600007106000074
:1000B0007106000071060000710600007106000064
:1000C0007106000071060000710600007106000054
:1000D0007106000071060000710600007106000044
:1000E0007106000071060000000000000000000022
:1000F00000000000390600007106000071060000D3
:100100007106000071060000710600007106000013
:100110007106000071060000710600007106000003
:1001200071060000710600007106000071060000F3
:1001300071060000710600007106000071060000E3
:1001400071060000710600007106000071060000D3
:1001500071060000710600007106000071060000C3
:1001600071060000710600007106000071060000B3
:1001700071060000710600007106000071060000A3
:100180007106000071060000710600007106000093
:100190007106000071060000710600007106000083
:1001A0007106000071060000710600007106000073
:1001B0007106000071060000710600007106000063
:1001C0007106000071060000710600007106000053
:1001D0007106000071060000710600007106000043
:1001E0007106000071060000710600007106000033
:1001F0007106000071060000710600007106000023
:100200007106000071060000710600007106000012
:100210007106000071060000710600007106000002
:1002200071060000710600007106000071060000F2
:1002300071060000710600007106000071060000E2
:1002400071060000710600007106000071060000D2
:1002500071060000710600007106000071060000C2
:100260007106000010B5054C237833B9044B13B167
:100270000448AFF300800123237010BD6400002008
:10028000000000001418000008B5034B1BB103491F
:100290000348AFF3008008BD0000000068000020A4
:1002A0001418000070B50D461646044610B1081E1D
:1002B00018BF01200549064B34229847236832466F
:1002C00029462046BDE87040184700BF741600005C
:1002D000850400004FF0E0236FF07F425A61052251
:1002E0001A617047044A1168034609B9034911604D
:1002F000106803441360704780000020D80001207C
:1003000038B50D46044610B1081E18BF01200A4931
:100310000A4B402298472046094B40F8045F294683
:100320009847002807DB4FF40043A382054B236165
:10033000054BE360002038BD8816000085040000EE
:10034000850A0000C10300008903000030B50C4697
:1003500085B0054610B1081E18BF0120B322074919
:10036000074B98472368019363680293A36803933C
:1003700001A9044B281D984705B030BD8816000020
:1003800085040000B90B00007FB50446003818BF93
:1003900001200E4615460749074BA3229847002324
:1003A000CDE9016301A9054B0395A4F10C00984721
:1003B00004B070BD88160000850400004D030000E5
:1003C0007FB50446003818BF01200E461546074980
:1003D000074B872298470023019301A9054B0296FA
:1003E000A4F10C000395984704B070BD8816000076
:1003F000850400004D030000014B1860014B1847B5
:1004000084000020D50200000A4A13889BB210B570
:1004100043F4A0631380084B9847084B9847084B58
:100420009847084B9847BDE81040074B40F6FF70CF
:10043000184700BF00400041290700008B0400005E
:100440002D0600008D0400004D040000C20707D5F2
:10045000094B0A4A1A6243F6FD7259681142FCD1EF
:10046000030707D5044B064ADA6243F6FD72596862
:100470001142FCD1704700BF001C00400701010081
:100480000501010000B900BE704770470C4B0D4AD2
:100490005A63DA6B12F0060FFBD14FF402629A63D3
:1004A000022283F83020064AD36B9807FCD4044B11
:1004B0001A6CD10702D41A6C9207F9D5704700BFA5
:1004C000001000404D0E01002DE9F8430E46154680
:1004D000044618B129B3101E18BF01201249134B4E
:1004E000134FF12298470834B9462046B8470028F0
:1004F000FBD0DFF844800027F15D2046C04720464E
:10050000C8470028FBD00137BD42F5D8002D094E61
:1005100008BF01252046B0470028FBD02846BDE88B
:10052000F8830846DAE700BFA4160000850400003F
:10053000670A0000710A0000590A00002DE9F8431B
:100540000E461546044618B1E9B1101E18BF012029
:100550000E490F4BDFF83C90DFF83C804FF4867279
:100560009847002708342046C8470028FBD020467B
:10057000C047F0550137BD42F5D8002D14BF2846BD
:100580000120BDE8F8830846E2E700BFA41600009A
:10059000850400007B0A00005F0A000038B50D46A4
:1005A000044610B1081E18BF01200749074B34222A
:1005B0009847074B294604F10800984718B9054B9E
:1005C0006360054B236038BDA4160000850400005D
:1005D000190A00003D050000C904000010B50446DA
:1005E000003818BF01200549054B5322984704F1F4
:1005F0000800044B9847002010BD00BFA41600005F
:1006000085040000450A000038B50D46044610B1C7
:10061000081E18BF01200349034B692298472C602C
:10062000002038BDA416000085040000014B012203
:100630005A717047000800400B4A937882B0DBB2D1
:100640000193019B990705D5084B1B6813B15068AE
:1006500002B01847019BDB0704D5044B5B680BB164
:10066000014AF4E702B07047000002418800002010
:10067000FEE7000018491948814210B50AD0184B0E
:10068000DA1C121A22F00302C41EA34238BF002251
:10069000144B9847144B1548DA1C121AC11E22F04D
:1006A0000302994288BF0022114B00219847114A4A
:1006B000114B22F07F029A60D3F8882042F4700236
:1006C000C3F88820BFF34F8FBFF36F8F0B4B984752
:1006D0000B4B9847FEE700BF1418000000000020F5
:1006E000640000205D0D0000D800002064000020A0
:1006F000790D00000000000000ED00E0150D000085
:100700000507000008B5044B9847044B9847044878
:10071000044B9847FEE700BF790C0000E10C000095
:10072000C0160000810C0000064B42F28E329A8205
:1007300000229A75DA75DA6902F47C52DA610122D4
:100740001A7470470014004000F01F0303F1824147
:1007500001F500415B0891F8C02003F1824302F0EB
:10076000FE0242F0010203F5004381F8C02093F835
:10077000B02010F0010F15BF02F00F0202F0F002DE
:1007800042F0300242F0030283F8B02070470000CC
:1007900010B5054C05493920A04723460449BDE85A
:1007A00010403820184700BF4907000003003900F7
:1007B00003003800064B4022C3F8DC204322C3F874
:1007C0008C20044A936943F400739361704700BF1F
:1007D000001C00400008004010B5054B05490648C4
:1007E0009847064B00229847BDE81040044B184735
:1007F000B507000000200141980000209D05000081
:100800009107000070B51B4C1B4D1C494FF0006355
:10081000C4F894304FF08046C4F88830184BC4F8C0
:10082000A8603B20C4F8A830A8474FF08063C4F804
:100830009430C4F88830134BC4F8A8601249C4F847
:10084000A8303A20A8474FF00053C4F884300F4B2B
:10085000C4F8A8300E4BC4F8A83094F8DD300D4928
:1008600003F0FB0384F8DD303D202B46BDE87040EB
:10087000184700BF008000414907000003003B000B
:10088000000800C0000400C003003A00000002405D
:10089000002002C003003D00064B4022C3F808219F
:1008A0004322C3F88C20044A136A43F00103136205
:1008B000704700BF001C00400008004010B5054B09
:1008C000054898474FF08641044B9847BDE81040D3
:1008D000034B184799080000A40000200103000002
:1008E000050800000148024B184700BF10E000E077
:1008F000F903000010B5054B9847054B9847054B89
:100900009847BDE81040044B184700BF0904000099
:10091000D9070000BD080000E5080000C3690B42CC
:10092000FCD17047C3690B42FCD170470268034B8E
:1009300022F0020202600321184700BF1D090000D7
:100940000268034B22F0020202600321184700BF35
:100950002509000070B50C4D06460FCD88B06C46D9
:100960000FC495E80F0084E80F006A46002352F890
:10097000041BB14202D1D8B208B070BD0133082BBC
:10098000F5D10020F8E700BFE016000038B51B4B9A
:1009900004469847022805D019491A4B40F24722CD
:1009A00000209847E369184D13F0010F0ED1032181
:1009B0002046A84723689B0703D5144B984702217C
:1009C000A8470523236003212046A847204601218C
:1009D000A8470F4B23600321A8474FF440336360BF
:1009E0001F21A8470B4BA3604FF61143A38100239F
:1009F000A373184684F8303038BD00BF5509000095
:100A0000C41600008504000025090000410900000B
:100A1000040010400200700070B5054600380C4616
:100A2000054B064918BF0120BB2298472C60204681
:100A3000034BBDE87040184785040000C416000051
:100A40008D0900000068036843F00203036003217E
:100A5000004B184725090000036899627047036836
:100A6000986AC0B270470368187E00F001007047B2
:100A70000368187EC0F3400070470368187EC0F317
:100A8000800070472DE9F843444B454D0746084622
:100A90000C469847042818BF0025002F5DD0201E63
:100AA00018BF01203F4E404940F63F12B047B046C4
:100AB000002D70D0E3693D4E13F0010F13D10321D7
:100AC0002046D5F80090B04723689B0709F01C0921
:100AD00003D5374B98470221B04749F00103236003
:100AE00003212046B04701212046B0472B68DFF89C
:100AF000C4903C6003F01C03082B30D12A4901202C
:100B000040F61D12C0472B6803EA09032360032146
:100B10002046B0476B6823F4083323F4107343F482
:100B2000003343F4107363601721B047AB6863620E
:100B30006B7B84F83030E369002BFCD16B6813F0D9
:100B4000070F0CBF012302233B71AB7BEA7B43EA17
:100B50000223FB800020BDE8F8833846A2E7124953
:100B6000012040F60912C0472B6803EA09032360FD
:100B700003212046B0476B6823F4383323F4107305
:100B800043F4003363601721B0472B7B23736B7BE7
:100B900084F83030D2E76FF00C00DCE75509000034
:100BA0001817000085040000C41600001D0900008D
:100BB0002D090000FCFEFFFF2DE9F843046890F8C2
:100BC00004802A4B0746201ED1E9006540F6A32287
:100BD00018BF0120894626499847E26912F00702AA
:100BE0003ED1244B032120469847236899073AD5E4
:100BF0001146237ED8B25B070FD48A4218D8C307A8
:100C000016D5FB8836B1B8F1010F33788CBF36F8B2
:100C1000023B01360132A3620AE0A36A3DB1B8F19A
:100C2000010F2B7085BF1B0A6B7001350235013136
:100C3000000607D4D9F808309342DAD88B42D8D8C6
:100C4000104606E04FF6FF736383802323766FF030
:100C50001200237E9B07FCD003232376BDE8F88394
:100C60006FF00300FAE76FF01300F7E78504000068
:100C7000C41600001D090000004B1847F5080000CD
:100C80000FB430B5C3B0114C469D2846A047FF288D
:100C900018D80F4B4FF48072002102A8984747AA3A
:100CA0000C4B0192294602A8984702A8A0470A4B7C
:100CB00082B202A91868094B984743B0BDE830409A
:100CC00004B070474FF0FF30F7E700BF890D000018
:100CD000790D0000C50D0000BC000020A502000039
:100CE00010B5064C0649074B20469847064B204650
:100CF0009847064B06489847002010BD98000020F2
:100D0000BC00002009060000DD050000810C000089
:100D10002917000070B50D4D0D4C641BA410002662
:100D2000A64209D10B4D0C4C00F064FD641BA410CD
:100D30000026A64205D170BD55F8043B9847013600
:100D4000EEE755F8043B98470136F2E7001800003B
:100D50000018000000180000041800000A44914226
:100D600000F1FF3300D1704710B511F8014B03F8C3
:100D7000014F9142F9D110BD02440346934200D184
:100D8000704703F8011BF9E7034613F8012B002A0B
:100D9000FBD1181A0138704700B59BB0009104913F
:100DA0006FF000410591029105490391694600F0F9
:100DB000CBF8009B00221A701BB05DF804FB00BF4B
:100DC0000802FFFF13460A46014602480068FFF783
:100DD000E3BF00BF0000002070477047F8B5CD1C8E
:100DE00025F0030508350C2D38BF0C25002D0646CF
:100DF00001DBA94203D90C2333600020F8BD00F0C9
:100E0000B1FB21490A6814469CB9204F3B6823B9BD
:100E10002146304600F02CFB38602946304600F071
:100E200027FB431C23D10C233360304600F0A0FB8A
:100E3000E3E723685B1B17D40B2B03D923601C4407
:100E4000256004E06368A2420CBF0B60536030462B
:100E500000F08EFB04F10B00231D20F00700C21AE6
:100E6000CCD01B1AA350C9E722466468CCE7C41C47
:100E700024F00304A042E3D0211A304600F0F8FA2F
:100E80000130DDD1CFE700BFC0000020C40000204A
:100E90002DE9F0478E689E4282460C4690461F46DA
:100EA00038D88A8912F4906F32D025680969A5EB89
:100EB0000109656905EB450505EBD57501334B4423
:100EC0006D109D4238BF1D46530531D52946FFF7A9
:100ED00085FF064650B90C23CAF80030A38943F0B9
:100EE0004003A3814FF0FF30BDE8F08721694A46F7
:100EF000FFF734FFA38923F4906343F08003A381B9
:100F0000266165614E44A5EB09052660A5603E4655
:100F1000BE4200D93E4632462068414600F008FBFA
:100F2000A36822689B1B3244A36022600020DBE799
:100F30002A4600F071FB06460028E1D1216950469F
:100F400000F01CFBC7E700002DE9F04F98468B89A5
:100F50001B069DB007460D4614460ED50B6963B9B6
:100F60004021FFF73BFF2860286120B90C233B603C
:100F70004FF0FF30D1E040236B6100230993202321
:100F80008DF82930CDF80C803023DFF8A8818DF85A
:100F90002A304FF0010923469A4613F8012B0AB173
:100FA000252AF9D1BAEB040B0BD05B462246294621
:100FB0003846FFF76DFF013000F0AA80099A5A44C5
:100FC00009929AF80030002B00F0A28000234FF025
:100FD000FF32CDE905230AF1010A049307938DF846
:100FE00053301A935446052214F8011B514800F05F
:100FF0004FFA049AD8B9D00644BF20238DF8533055
:10100000110744BF2B238DF853309AF800302A2B58
:1010100015D0079A544600204FF00A0C214611F8CB
:10102000013B303B092B4ED9B0B1079214E0A0EB45
:10103000080309FA03F313430493A246D2E7039B80
:10104000191D1B680391002BBBBF5B4242F00202DB
:1010500007930793B8BF049223782E2B0CD16378A3
:101060002A2B35D1039B1A1D1B680392002BB8BF96
:101070004FF0FF3302340593DFF8C8A02178032234
:10108000504600F005FA40B14023A0EB0A0003FAF5
:1010900000F0049B03430134049314F8011B264819
:1010A0008DF82810062200F0F3F9002838D0234BE1
:1010B0001BBB039B073323F0070308330393099BF0
:1010C0003344099367E70CFB02320C460120A5E785
:1010D00000230134059319464FF00A0C204610F8FE
:1010E000012B303A092A03D9002BC5D00591C3E75B
:1010F0000CFB012104460123F0E703AB00932A46D1
:101100000F4B04A93846AFF30080421C0646D6D1E7
:10111000AB895B063FF52CAF09981DB0BDE8F08F99
:1011200003AB00932A46064B04A9384600F07AF830
:10113000EBE700BFC0170000CA1700000000000066
:10114000910E0000C61700002DE9F047164699469B
:101150008A680B69DDF820809342B8BF134633607C
:1011600091F8432007460C460AB1013333602368E7
:10117000990642BF336802333360256815F00605CF
:1011800006D104F1190AE36832689B1AAB4226DCE7
:1011900094F84320131E226818BF012392062BD413
:1011A00004F1430249463846C04701301ED0236847
:1011B000E568326803F00603042B08BFAD1AA36884
:1011C00022690CBF25EAE57500259342C4BF9B1A2E
:1011D000ED1800261A34B5421AD1002008E0012388
:1011E000524649463846C047013003D14FF0FF30E0
:1011F000BDE8F0870135C6E7E1185A1C302081F8B8
:101200004300224494F8451082F843100233C7E7A4
:101210000123224649463846C0470130E6D0013610
:10122000D9E700002DE9FF470C469146277E0C992F
:10123000782F80469A4604F1430207D8622F0AD8D5
:10124000002F00F0D880582F00F0A38004F1420650
:1012500084F842703AE0A7F16303152BF6D801A099
:1012600050F823F0BD120000D11200004D12000012
:101270004D1200004D1200004D120000D11200006E
:101280004D1200004D1200004D1200004D120000E2
:10129000DD13000001130000BF1300004D12000019
:1012A0004D120000FF1300004D120000011300005A
:1012B0004D1200004D120000C71300000B681A1DEC
:1012C0001B680A6004F1420684F842300123A3E05F
:1012D000256808682E0600F104030AD505680B602E
:1012E000002D03DA2D236D4284F843305E480A2333
:1012F00019E015F0400F05680B6018BF2DB2EFE73D
:101300000B682568181D0860280601D51D6802E0D5
:101310006906FBD51D8854486F2F0CBF08230A238C
:10132000002184F843106668A660002EA2BF2168E1
:1013300021F0040121600DB9002E4DD01646B5FBF9
:10134000F3F103FB1157C75D06F8017D2F46BB4241
:101350000D46F4D9082B0BD12368DF0708D5236984
:1013600061689942DEBF302306F8013C06F1FF3682
:10137000921B2261CDF800A04B4603AA21464046AD
:10138000FFF7E2FE01304CD14FF0FF3004B0BDE872
:10139000F087354884F8457023680E681F0656F8B4
:1013A000045B0E6014D5D90744BF43F020032360CB
:1013B0001DB9236823F0200323601023B0E72368BE
:1013C00043F0200323607823284884F84530E3E77E
:1013D0005E0648BFADB2E6E71646BBE70B68266877
:1013E00060691D1D0D6035061B6801D5186002E09F
:1013F0007106FBD51880002323611646BAE70B68F7
:101400001A1D0A601E6862680021304600F040F82C
:1014100008B1801B606063682361002384F8433057
:10142000A8E72369324649464046D0470130ABD051
:1014300023689B0713D4E068039B9842B8BF184603
:10144000A4E70123324649464046D04701309BD0AD
:101450000135E36803995B1AAB42F2DCEBE7002548
:1014600004F11906F5E700BFD1170000E2170000EC
:1014700038B5064D0023044608462B60FEF732FFC0
:10148000431C02D12B6803B1236038BDD400002077
:1014900001F0FF01102A2BDB10F0070F08D010F825
:1014A000013B013A8B422DD010F0070F42B3F6D129
:1014B000F0B441EA012141EA014122F007047FF042
:1014C00000070023F0E80256083C85EA010586EA99
:1014D000010685FA47F5A3FA87F586FA47F6A5FAD5
:1014E00087F68EB9EED1F0BC01F0FF0102F00702E1
:1014F00032B110F8013B013A83EA010313B1F8D18C
:101500000020704701387047002D06BF354603386C
:10151000073815F0010F07D1013015F4807F02BFA5
:10152000013015F4C03F0130F0BC0138704700BFF6
:10153000884210B501EB020402D98442234607D841
:10154000431EA14208D011F8012B03F8012FF8E740
:10155000024401468A4200D110BD13F8014D02F841
:10156000014DF7E70148FFF737BC00BFCC00002072
:101570000148FFF732BC00BFCC00002038B505465B
:10158000002945D051F8043C0C1F002BB8BFE418CB
:10159000FFF7E8FF1F4A1368104633B96360146011
:1015A0002846BDE83840FFF7E3BFA3420BD92168C6
:1015B0006218934204BF1A685B68636004BF5218E4
:1015C00022600460ECE71A465B680BB1A342FAD9CB
:1015D00011685018A0420BD1206801445018834272
:1015E0001160DDD118685B68536001441160D7E772
:1015F00002D90C232B60D3E7206821188B4204BF4B
:1016000019685B68636004BF091821605460C7E70C
:1016100038BD00BFC0000020F8B5074614460E468E
:1016200021B9BDE8F8401146FFF7D8BB22B9FFF752
:10163000A5FF25462846F8BD00F014F8A0420FD2B9
:1016400021463846FFF7CAFB05460028F2D031464E
:101650002246FFF783FB31463846FFF78FFFE9E765
:101660003546E7E751F8043C181F002BBCBF0B5868
:10167000C01870472E2E2F68616C2F7372632F680D
:10168000616C5F696F2E63002E2E2F68616C2F7363
:1016900072632F68616C5F7370695F6D5F73796EE1
:1016A000632E63002E2E2F68616C2F7372632F6878
:1016B000616C5F75736172745F73796E632E630022
:1016C00048690A002E2E2F68706C2F736572636F45
:1016D0006D2F68706C5F736572636F6D2E630000B1
:1016E0000030004000340040002001410040014132
:1016F000000000430004004300080043000C0043C6
:1017000000000000000000000000000000000000D9
:1017100000000000000000000C003000000002008B
:1017200000000000FE00FF01044465627567204967
:101730006E697469616C697A65640A0041737365E6
:101740007274204661696C757265206174206C69E1
:101750006E652025642C2025733A2025730A00002D
:101760000000000000000000000000000000000079
:101770000000000000000000000000000000000069
:101780000000000000000000000000000000000059
:101790000000000000000000000000000000000049
:1017A0000000000000000000000000000000000039
:1017B0000000000000000000000000000000000029
:1017C000232D302B2000686C4C006566674546472A
:1017D00000303132333435363738394142434445AD
:1017E000460030313233343536373839616263641C
:1017F00065660000F8B500BFF8BC08BC9E4670479F
:1018000089020000F8B500BFF8BC08BC9E467047CE
:04181000650200006D
:10181400040000200000000080170000A017000052
:10182400601700000000000000000000000000003D
:1018340000000000000000000000000000000000A4
:101844000000000000000000000000000000000094
:101854000000000000000000000000000000000084
:101864000000000000000000000000000000000074
:041874000000000070
:00000001FF
